:020000020000FC
:020000004FC0EF
:0200340015C0F5
:100060000FB704C00FBF10E91AB918952CB12F3F74
:1000700019F4E0E6F0E0F6CF2193E23611F4E0E681
:1000800001C0F0CF10916000107F1030109160001F
:100090001F70C0E8D0E0C10F109161001883E2CF5B
:1000A00031E03EBF3FE53DBF37E639B930E93AB907
:1000B0003EE830BD30936000309361003FE73093FD
:1000C000800030938100309382003093830030931E
:1000D00084003093850030938600309387003093FE
:1000E00088003093890030938A0030938B003093DE
:1000F0008C0030938D0030938E0030938F003FEF53
:100100003ABB34BB30E03BBB35BB789440E052E0B7
:10011000609180007091810032D044E058E060919D
:100120008200709183002BD040E150E26091840006
:100130007091850024D040E450E860918600709171
:1001400087001DD040E850E46091880070918900DC
:1001500040D040E250E160918A0070918B0039D02C
:1001600048E054E060918C0070918D0032D042E004
:1001700050E060918E0070918F002BD0C7CF3BB3C1
:10018000342B352B3BBB4FD080E0861731F43BB38B
:100190004095342340953BBB06C0000000000000A2
:1001A000000000000000871731F43BB35095352361
:1001B00050953BBB06C0000000000000000000009E
:1001C000000032E100003A95E9F783958F3FE9F6A8
:1001D000089535B3342B352B35BB25D080E08617F9
:1001E00031F435B340953423409535BB06C000004B
:1001F00000000000000000000000871731F435B354
:1002000050953523509535BB06C000000000000016
:1002100000000000000032E100003A95E9F7839504
:100220008F3FE9F6089537E004D03A953030E1F792
:1002300008953F933FE90000000000000000000027
:0C024000000000003A95B9F73F910895C6
:00000001FF
